:100000000C947B030C943E1C0C946B1C0C94E72109
:100010000C940B220C942F220C94A3030C94A30396
:100020000C94A3030C94A3030C94A3030C94A303B8
:100030000C94A3030C94A3030C94A3030C94A303A8
:100040000C94981C0C94A3030C94B91E0C94FC1EE5
:100050000C94A3030C94A3030C94A3030C94A30388
:100060000C94472A0C94A303A518B818D218E518C5
:10007000FC18281930193819401947194719471918
:100080004719471947194719471947194719471970
:100090004719471947194719471947194719471960
:1000A0004719471947194719A518B118B818D21890
:1000B000E518FC180F1917191F19084AD73B3BCE32
:1000C000016E84BCBFFDC12F3D6C74319ABD568357
:1000D0003DDA3D00C77F11BED9E4BB4C3E916BAA0F
:1000E000AABE000000803F05A84CCDB2D44EB9385E
:1000F00036A9020C50B9918688083CA6AAAA2ABE45
:10010000000000803F002075532F68002075532F9A
:100110006800206D532F68002043504D006B435002
:100120004D002530356C642E2530346C640025304C
:10013000346C642E2530346C640024504D544B31A3
:1001400030342A3337004E4F205344204341524429
:100150002F20475053207265736574002530326438
:100160002F2530326420253032643A253032643A0B
:10017000253032640057726F6E67206D6F646520A2
:10018000210075530044733D0075532F6820004DC6
:10019000783D0042712F6D32006B42712F6D32003D
:1001A0006D42712F6D320043504D20006B43504D16
:1001B00020002D2D006B6D002042712F6D3200202C
:1001C0007553762F68005E004E6F20475053002510
:1001D00030326468253032646D002A2558002A3098
:1001E0002558002425732C253034642C25303264A6
:1001F0002D253032642D2530326454253032643A56
:10020000253032643A253032645A2C256C642C2512
:100210006C642C256C642C25632C25732C25632C95
:1002200025732C25632C25732C25632C25642C2504
:100230006C64002530346425303264253032642EFD
:100240006C6F67006E616E6F0A2320646561647471
:10025000696D653D6F6E0A00312E342E310023200A
:100260004E4557204C4F470A2320666F726D6174CC
:100270003D0024504D544B3330312C322A32450D41
:100280000A0024504D544B3331332C312A32450D62
:100290000A0024504D544B3232302C313030302A49
:1002A00031460024504D544B3331342C302C312CFA
:1002B000302C312C302C302C302C302C302C302C5D
:1002C000302C302C302C302C302C302C302C302C4E
:1002D000302A3238002325303464004D6F646520A5
:1002E0003D25640043504D00416C61726D3D2564B5
:1002F00000252500426174746572793D20253032F5
:100300006400476569676965204E616E6F202573DB
:1003100000726561642025732030202564004A50F6
:100320004E00000000070002010000030406000068
:1003300000000000000001020408102040800102BB
:10034000040810200102040810200404040404041A
:100350000404020202020202030303030303000077
:1003600000002300260029000000000025002800CE
:100370002B0000000000240027002A0000C201001A
:10038000010005000500030000E1000001000F006E
:100390000F000D0000960000020019001A0017005F
:1003A000127A00000700200021001D00807000006C
:1003B0000B00230023002000004B00001400370036
:1003C00037003400403800001E004B004B0048004E
:1003D000802500003200720072007000C012000020
:1003E0006E00E900E900E60060090000E500D801C0
:1003F000D801D501B0040000D301B403B403B103A4
:1004000058020000B4036707670762072C01000069
:100410006707DD0EDD0EDA0E000000000000005F51
:1004200000000007000700147F147F14242A7F2A8D
:10043000122313086462364956205000080703004F
:10044000001C2241000041221C002A1C7F1C2A089B
:10045000083E0808008070300008080808080000FE
:1004600060600020100804023E5149453E00427F72
:10047000400072494949462141494D331814127FC1
:100480001027454545393C4A494931412111090761
:100490003649494936464949291E000014000000E2
:1004A00040340000000814224114141414140041B4
:1004B00022140802015909063E415D594E7C121171
:1004C000127C7F494949363E414141227F414141A9
:1004D0003E7F494949417F090909013E4141517324
:1004E0007F0808087F00417F41002040413F017F95
:1004F000081422417F404040407F021C027F7F045D
:1005000008107F3E4141413E7F090909063E4151A5
:10051000215E7F09192946264949493203017F0195
:10052000033F4040403F1F2040201F3F4038403F96
:10053000631408146303047804036159494D4300AC
:100540007F4141410204081020004141417F0402E3
:10055000010204404040404000030708002054547A
:1005600078407F2844443838444444283844442858
:100570007F385454541800087E090218A4A49C78AB
:100580007F0804047800447D40002040403D007F07
:100590001028440000417F40007C047804787C08E7
:1005A0000404783844444438FC18242418182424BB
:1005B00018FC7C08040408485454542404043F44A0
:1005C000243C4040207C1C2040201C3C4030403CCF
:1005D00044281028444C9090907C4464544C44002F
:1005E0000836410000007700000041360800020193
:1005F00002040200407A10F35A00A0724E1809005B
:1006000010A5D4E80000E87648170000E40B540277
:100610000000CA9A3B000000E1F5050000809698B2
:1006200000000040420F000000A086010000001002
:100630002700000000E80300000000640000000044
:10064000000A00000000000100000000002C76D825
:1006500088DC674F0823DFC1DFAE59E1B1B796E50B
:10066000E3E453C63AE651997696E8E6C28426EB6F
:10067000898C9B62ED407C6FFCEFBC9C9F40F2BA82
:10068000A56FA5F490055A2AF75C936B6CF9676D1A
:10069000C11BFCE0E40D47FEF520E6B500D0ED906F
:1006A0002E0300943577050080841E080000204E3C
:1006B0000A000000C80C333333330F986E128311D5
:1006C00041EF8D2114893BE65516CFFEE6DB18D1AC
:1006D000844B381BF77C1D901DA4BBE4242032847E
:1006E000725E228100C9F124ECA1E53D27009D0541
:1006F000B21FA829D20511241FBECFEFD8E0DEBF5C
:10070000CDBF13E0A0E0B1E0EAE4FAE602C0059054
:100710000D92AC3FB107D9F728E0ACEFB3E001C0D0
:100720001D92A933B207E1F716E0C4EFD6E004C08A
:100730002297FE010E94122FCE3ED107C9F70E94D8
:1007400072200C9418350C9400008EE00E94751DE8
:10075000BC01882777FD8095982F0E94DD2C20E032
:1007600030E040E85AE30E94F62D20E030E040E21D
:1007700051E40E94F62D24EB35EC4AEC5DE30E9437
:10078000422C0895A0E0B0E0E8ECF3E00C94302FA8
:10079000982E6A017B01B22EA32ECB01BA0120EA6A
:1007A00036E841E050E00E94EE2EE901142F052FBB
:1007B00060EA76E881E090E00E94CA2EA7019601E7
:1007C000261B370B480B590BCA01B9012AE030E050
:1007D00040E050E00E94EE2E9920D1F05F934F93BD
:1007E0003F932F930F931F93DF93CF938EE291E06C
:1007F0009F938F93AF92BF920E9412304DB75EB716
:10080000445F5F4F0FB6F8945EBF0FBE4DBF18C078
:100810005F934F933F932F930F931F93DF93CF9348
:1008200082E291E09F938F93AF92BF920E94123029
:100830008DB79EB70C960FB6F8949EBF0FBE8DBFB6
:10084000CDB7DEB7EBE00C944C2F8F929F92AF9216
:10085000BF92CF92DF92EF92FF920E94DB2C20E8B2
:1008600036E948E15BE40E94422C4B015C010E94A6
:10087000AA2C882777FD8095982F0E94DD2C6B018C
:100880007C019B01AC01C501B4010E94742B20E0E6
:1008900030E040E752E40E94422C20E030E048EC97
:1008A00052E40E94F62DA70196010E94752BFF903D
:1008B000EF90DF90CF90BF90AF909F908F90089572
:1008C0004F925F926F927F928F929F92AF92BF9260
:1008D000EF92FF920F931F932B013C0149015A01A4
:1008E000A70160E070E086E096E00E94F52562E0F6
:1008F00086E096E00E94FB2580910701863549F449
:1009000041E050E060E070E086E096E00E9407265B
:1009100006C061E070E086E096E00E94012680E279
:10092000E2E0F5E0DF011D928A95E9F7809131045C
:1009300090913204A0E0B0E088159905AA05BB05A6
:1009400040F4ACE0B0E0A30192010E94162F4B01ED
:100950005C01C501B401002309F447C0B0E18B1666
:10096000B7E29B06A104B10440F10E94DB2C20E019
:1009700030E04AE754E40E94422C02E215E023E012
:1009800044E00E94832F43E050E0B80182E095E00C
:100990000E94D92FE2E0F5E001900020E9F73297BC
:1009A00080818E3209F4108262E075E086E096E084
:1009B0000E9441208DE191E0A1C00E94DB2C02E267
:1009C00015E020E040E00E94832FB80186E096E029
:1009D0000E94412088E191E09F938F93C8019F93EB
:1009E0000F930E941230B80193C00E94DB2C20911B
:1009F000290430912A0440912B0450912C040E9428
:100A0000422C4B015C0120E030E04AE754E40E94B4
:100A1000EB2D87FD28C020E030E04AE754E4C50113
:100A2000B4010E94422C02E215E022E044E00E9460
:100A3000832F45E050E0B80182E095E00E94D92F75
:100A4000E2E0F5E001900020E9F7329780818E32F4
:100A500009F4108262E075E086E096E00E94412091
:100A600082E191E04BC020E030E040E251E4C5017A
:100A7000B4010E94EB2D02E215E087FD20C022E0C8
:100A800044E0C501B4010E94832F45E050E0B80165
:100A900082E095E00E94D92FE2E0F5E0019000208D
:100AA000E9F7329780818E3209F4108262E075E0B6
:100AB00086E096E00E9441208CE091E01FC023E098
:100AC00044E0C501B4010E94832F46E050E0B80124
:100AD00082E095E00E94D92FE2E0F5E0019000204D
:100AE000E9F7329780818E3209F4108262E075E076
:100AF00086E096E00E94412086E091E09F938F93EC
:100B000082E295E09F938F930E94123062E275E03B
:100B100086E096E00E9441200F900F900F900F907A
:100B20001F910F91FF90EF90BF90AF909F908F908B
:100B30007F906F905F904F900895EF92FF920F9388
:100B40001F938CE0E82E0DE02BE04AE069E086E0A0
:100B500096E00E94B42620E045E066E086EE94E050
:100B60000E94A12261E081E794E00E94AF1520E09D
:100B700047E068E085E594E00E94A12294E6E92E32
:100B8000F12C02E415E028E034E040E154E066EEA8
:100B900074E08EEF93E00E9455121F910F91FF9029
:100BA000EF90089585E594E00E94A32386EE94E0FB
:100BB0000E94A32308951F93CF93DF93182FC0E0C3
:100BC000D0E0219686EE94E00E94B820892B51F463
:100BD0006AE070E080E090E00E94111DC83CD10501
:100BE00081F712C086EE94E00E947F20112319F055
:100BF0002EE330E002C02CE330E08217930741F788
:100C000081E0C83CD10509F480E0DF91CF911F91CC
:100C100008950F931F93CF93DF9362E083E00E94C8
:100C2000BB1D61E082E10E94BB1D60E083E10E9488
:100C3000BB1D40E855E260E070E08AE496E00E9467
:100C4000371F8EEF93E00E94A81240E855E260E063
:100C500070E086EE94E00E94D12261E084E00E9480
:100C6000BB1D86EE94E00E94F22060E084E00E94CA
:100C7000F41D64E670E080E090E00E94111D61E0E8
:100C800084E00E94F41D81E00E94DB05811104C014
:100C900081E08093EC0503C081E08093E5048091BE
:100CA000E504882331F06AE073E08EEF93E00E9460
:100CB0002B1348E853E160E070E080E090E00E9490
:100CC000D9110E94F41140E855E260E070E085E53A
:100CD00094E00E94D12285E594E00E94F220C2E4D3
:100CE000D5E014E6FE01812F11928A95E9F783EA97
:100CF00092E09F938F93DF93CF930E941230BE01B7
:100D000085E594E00E946020FE01812F11928A9572
:100D1000E9F782E992E09F938F93DF93CF930E944C
:100D20001230BE0185E594E00E946020FE01812F13
:100D300011928A95E9F782E892E09F938F93DF936F
:100D4000CF930E941230BE0185E594E00E9460209E
:100D5000FE0111921A95E9F782E792E09F938F9333
:100D6000DF93CF930E941230BE0185E594E00E948C
:100D70006020C8E0D4E0EDB7FEB770960FB6F894E7
:100D8000FEBF0FBEEDBF68EC70E08B010F5F1F4F21
:100D900088E797E00E94AB238993003D110511F08D
:100DA000B801F3CF83E00E94721D4CE362E086E05D
:100DB00096E00E94352786E096E00E94482868EE7B
:100DC00073E080E090E00E94111D86E096E00E94B2
:100DD000C52661E070E086E096E00E94012661E0B1
:100DE00086E096E00E94FB2587E193E09F938F9336
:100DF00082E093E09F938F93C2E2D5E0DF93CF939D
:100E00000E94123009900020E9F7C252D54026E036
:100E10002C9FC0012D9F900D112460E870E0681B8D
:100E2000790B7695679540E050E086E096E00E9469
:100E3000F5250F900F900F900F900F900F908091CD
:100E40001404811103C06DE173E002C06FE173E02F
:100E500086E096E00E94412062E275E086E096E03E
:100E60000E94412048E050E068E070E086E096E0B3
:100E70000E94F5250E94A50320E030E040EF51E4F8
:100E80000E94742B20E030E048E451E40E94F62DEB
:100E90000E94AA2C6C5E7F4F77FD06C065367105F7
:100EA0002CF064E670E002C061E070E07F936F9325
:100EB00084EF92E09F938F93C2E2D5E0DF93CF93CC
:100EC0000E941230BE0186E096E00E94412081EF30
:100ED00092E09F938F93DF93CF930E941230BE01D5
:100EE00086E096E00E94412040E150E067E370E038
:100EF00086E096E00E94F525809132048F938091E0
:100F000031048F9388EE92E09F938F93DF93CF937A
:100F10000E941230BE0186E096E00E94412084EEDD
:100F200092E09F938F93DF93CF930E941230BE0184
:100F300086E096E00E94412040E150E068E070E0E9
:100F400086E096E00E94F52580913C041F928F93E5
:100F50008BED92E09F938F93DF93CF930E9412309B
:100F6000BE0186E096E00E94412061E086E096E0C6
:100F70000E94FB2548E050E065E570E086E096E0E1
:100F80000E94F525809127048F93809126048F93EA
:100F900085ED92E09F938F93DF93CF930E94123061
:100FA000EDB7FEB7B0960FB6F894FEBF0FBEEDBF1B
:100FB000BE0186E096E00E94412061E086E096E076
:100FC0000E94FB25809116048823F9F0E6E1F4E005
:100FD00001900020E9F7E751F44026E02E9FC00180
:100FE0002F9F900D112460E870E0681B790B7695B7
:100FF000679548E150E086E096E00E94F52566E1BD
:1010000074E086E096E00E94412086E096E00E942F
:10101000482868E273E280E090E00E94111DDF91B1
:10102000CF911F910F910895A4E2B0E0EAE1F8E0BA
:101030000C94292F83E10E94751D853F91401CF07F
:101040001092140407C081E08093140460E082E1F0
:101050000E94F41D0E94A50320E030E040EF51E41F
:101060000E94742B0E94AA2C161617064CF068EEEC
:1010700073E080E090E00E94111D81E080931404F1
:1010800085E594E00E94F2200E94E21C6B017C0145
:101090000E94E21C97018601061B170B280B390BD7
:1010A000C616D706E806F90618F0D901C80106C029
:1010B000D901C80180959095A095B095883E934040
:1010C000A105B105A0F40E940712892B81F485E5E2
:1010D00094E00E94B820892BD9F285E594E00E9423
:1010E0007F20682F81E794E00E945019F0CF0E9482
:1010F0000712892B11F40C94C1110E944C126D8BB4
:101100007E8B8F8B988F0E94F4118091B8059091FF
:10111000B905A091BA05B091BB05FC01EE0FFF1F08
:10112000EE0FFF1FE454FA4F2D893E894F89588DE9
:101130002083318342835383BC01CD016F5F7F4F96
:101140008F4F9F4F2CE030E040E050E00E94EE2EA9
:101150006093B8057093B9058093BA059093BB0569
:10116000ECEBF5E060E070E0CB0101911191219191
:101170003191600F711F821F931F35E0EC3EF30722
:10118000A1F70E94DB2C6B017C0122EB35EC4CEFCC
:1011900055E30E94F62D9B01AC0160E070E080E811
:1011A0009FE30E94742B9B01AC01C701B6010E9412
:1011B000422C0E94AF2C2B013C018091B4059091F0
:1011C000B505A091B605B091B7052D893E894F8927
:1011D000588D820F931FA41FB51F8093B405909361
:1011E000B505A093B605B093B7058091AC05909175
:1011F000AD05A091AE05B091AF050596A11DB11D3D
:101200008093AC059093AD05A093AE05B093AF0568
:101210008091B0059091B105A091B205B091B30550
:1012200084159505A605B70540F44092B005509287
:10123000B1056092B2057092B30580910804909157
:101240000904A0910A04B0910B042D893E894F89AD
:10125000588D820F931FA41FB51F8093080490938D
:101260000904A0930A04B0930B0460910C047091DC
:101270000D0480910E0490910F046B5F7F4F8F4F90
:101280009F4F60930C0470930D0480930E04909311
:101290000F0420E13EE040E050E00E94EE2E672B7C
:1012A000682B692B81F08091A6059091A7058C3061
:1012B0009105F4F426E52093070101969093A70584
:1012C0008093A6051FC008E014E068EC70E0D80128
:1012D0004D918D017B01BFEFEB1AFB0A88E797E088
:1012E0000E94AF23E0EDEE16F104E9F2B701EFCF73
:1012F000411451046104710411F486E501C081E4D4
:10130000809307018091EC058111ADC080910601A9
:10131000813409F0A8C08DED97E09E838D831A8AF1
:10132000198A188A1F861D8619869E012F5F3F4FD6
:101330004901AE01475F5F4F5A01CE010D966C0126
:10134000DE011F967D018E01005F1F4F205F3F4F22
:10135000475F5F4FBE016B5F7F4F81E794E00E9464
:101360001F1B89819A81AB81BC818F3F9F4FAF4FFB
:10137000BF4F09F478C089891F928F938A891F9281
:101380008F93809127048F93809126048F9383E31A
:1013900092E09F938F938DEE95E09F938F930E94A1
:1013A00012300FB6F894DEBF0FBECDBF81E0809340
:1013B000EC0586EE94E00E94F22068E273E086EE8F
:1013C00094E00E9441206DEE75E086EE94E00E946C
:1013D00041206DE086EE94E00E94792180E00E9439
:1013E000DB05811112C060E084E00E94F41D64E618
:1013F00070E080E090E00E94111D61E084E00E94B6
:10140000F41D81E00E94DB05D8CF8EE592E09F932A
:101410008F9302E215E01F930F930E941230B801E0
:1014200086EE94E00E94412088E592E09F938F939E
:101430001F930F930E941230B80186EE94E00E9431
:10144000412084E492E09F938F931F930F930E9417
:101450001230B80186EE94E00E9441200FB6F89455
:10146000DEBF0FBECDBF84E6E2E4F5E0DF011D92F2
:101470008A95E9F78DED97E09E878D871C8A1B8AF8
:101480001A8A198A188A1F8619861A861B861C864C
:101490001D821E821F8218868CE0E9E4F4E0DF01E1
:1014A000282F1D922A95E9F7EDE3F4E0DF011D9264
:1014B0008A95E9F780E2E2E2F5E0DF011D928A9584
:1014C000E9F7FE0131964F019E01215F3F4F59011F
:1014D000AE01405F5F4F6A01CE0141967C018E01F3
:1014E0000E5E1F4F2C5F3F4F4C5F5F4FBE01635F2F
:1014F0007F4F81E794E00E941F1B89819A81AB8115
:10150000BC818F3F9F4FAF4FBF4F51F48CED97E0A1
:101510009E878D871C8A1B8A1A8A198A188A1F86B9
:101520009E012F5F3F4FAE014B5F5F4FBE01675F74
:101530007F4F81E794E00E948F1A8091D904811136
:1015400002C086E501C081E48093060181E794E052
:101550000E94C61B6BA37CA31C0181E794E00E9440
:10156000FC1B6B017C012091B1043091B2043AA3C1
:1015700029A38090A9049090AA04A090AB04B090F5
:10158000AC0489859A85AB85BC85B7FF0EC0B09544
:10159000A095909581959F4FAF4FBF4F89879A87B0
:1015A000AB87BC8733E53D8F02C04EE44D8F8D8104
:1015B0009E81AF81B885B7FF0EC0B095A09590957C
:1015C00081959F4FAF4FBF4F8D839E83AF83B88769
:1015D00057E5598F02C085E4898F89859A85AB8547
:1015E000BC858F3FE9EC9E07EAE9AE07EBE3BE0757
:1015F00019F0AC01BD0104C040E050E060E070E0D3
:1016000029E434E081E00E94C2038D819E81AF8194
:10161000B8858F3FF9EC9F07FAE9AF07FBE3BF07F7
:1016200019F0AC01BD0104C040E050E060E070E0A2
:101630002DE334E080E00E94C2032091B103309199
:10164000B2034091B3035091B4036BA17CA1C101DB
:101650000E943B2C811105C0F0E0E0E050E030E05A
:1016600004C0FBA1ECA1522D332D02E215E022E0D3
:1016700040E06F2F7E2F852F932F0E94832F84E6CB
:10168000E2E4F5E0DF011D928A95E9F7BFEF8B16E2
:101690009B06AB06BB0629F420E030E040E050E0BA
:1016A00002C09401A501E9A1FAA1EF3FF10519F4E7
:1016B00080E090E002C089A19AA15F934F933F938D
:1016C0002F939F938F93809106011F928F9382E2B5
:1016D00095E09F938F931F92F98DFF938DE394E094
:1016E0009F938F931F922D8D2F9389E494E09F9366
:1016F0008F93809107011F928F938091B7058F93ED
:101700008091B6058F938091B5058F938091B40534
:101710008F93388D3F934F894F935E895F938D8967
:101720008F937F926F925F924F9288891F928F93CF
:1017300089891F928F938A891F928F938B891F9219
:101740008F938C891F928F938E858F938D858F9326
:10175000809127048F93809126048F9380E393E0F8
:101760009F938F9383EE91E09F938F9302E415E014
:101770001F930F930E941230F80101900020E9F7A7
:101780003197E254F540FF278F010E5B1A4FD801C5
:101790001C926091430584E495E00FB6F894DEBF97
:1017A0000FBECDBF2FEF3FEF22543540A901480FA8
:1017B000591F4E175F072CF4DC014D91CD016427B2
:1017C000F5CF603128F41F926F938EED91E004C045
:1017D0001F926F938AED91E09F938F931F930F93C6
:1017E0000E9412300F900F900F900F900F900F905B
:1017F0008091D904882309F4AFC069857A858B85E7
:101800009C850E942504698F7A8F8B8F9C8F6D81B8
:101810007E818F8198850E9425046D8F7E8F8F8FAA
:1018200098A320E030E040EA50E4C701B6010E94EE
:10183000EB2D181624F019E1812E912C03C0B5E090
:101840008B2E912C20E030E040E251E4C701B6013C
:101850000E94EB2D18161CF4AAE08A2E912C20E091
:1018600030E040E751E4C701B6010E94EB2D1816A5
:101870001CF4F4E18F2E912C809108018823D9F07B
:10188000298D3A8D4B8D5C8D2093FE053093FF059D
:1018900040930006509301068D8D9E8DAF8DB8A1AB
:1018A0008093020690930306A0930406B093050666
:1018B0001092080151C0A0900206B0900306C0909B
:1018C0000406D0900506E090FE05F090FF0500911B
:1018D0000006109101062D8D3E8D4F8D58A1698D0A
:1018E0007A8D8B8D9C8D0E94CD190E94AA2CAA24E2
:1018F00097FCA094BA2C86169706A806B90660F540
:101900000091FA051091FB052091FC053091FD0531
:10191000060F171F281F391F0093FA051093FB05A8
:101920002093FC053093FD05298D3A8D4B8D5C8D00
:101930002093FE053093FF05409300065093010667
:101940008D8D9E8DAF8DB8A1809302069093030676
:10195000A0930406B093050686E096E00E94C52693
:10196000809114048111B8C18090AC059090AD05B0
:10197000A090AE05B090AF05C501B40120E13EE0F6
:1019800040E050E00E94EE2E69017A013093AB05F1
:101990002093AA0524ECA60124038001259F100DA5
:1019A0001124C501B4012CE330E040E050E00E9476
:1019B000EE2E020F131F1093A9050093A8051F9385
:1019C0000F93DF92CF928FEC91E09F938F9382E2FF
:1019D00095E09F938F930E94123048E150E06CE5B0
:1019E00070E086E096E00E94F52561E086E096E0F2
:1019F0000E94FB2561E070E086E096E00E940126EF
:101A000062E275E086E096E00E9460200FB6F894EE
:101A1000DEBF0FBECDBF80910701813421F48091DC
:101A2000D9048111A7C460E082E10E94F41DE12C79
:101A3000F12C01E0A30192016D897E898F89988D37
:101A40000E94600461E070E086E096E00E9401265A
:101A500061E086E096E00E94FB258091D904811127
:101A600025C048E050E06CE570E086E096E00E941A
:101A7000F52541E050E060E070E086E096E00E94ED
:101A8000072688EC91E09F938F9382E295E09F93E5
:101A90008F930E94123062E275E086E096E00E9429
:101AA00060200F900F900F900F9033C061E070E0B6
:101AB00086E096E00E94012648E050E06EE670E085
:101AC00086E096E00E94F5259AA19F93A9A1AF9385
:101AD00086E393E09F938F9302E215E01F930F93A9
:101AE0000E94F02FB80186E096E00E94412086EC2B
:101AF00091E09F938F931F930F930E941230B80130
:101B000086E096E00E9460200FB6F894DEBF0FBE1C
:101B1000CDBF61E070E086E096E00E94012640E1E2
:101B200050E060E070E086E096E00E94F52580914C
:101B3000150481111CC0C301B2010E94DB2C20914D
:101B4000290430912A0440912B0450912C040E94C6
:101B5000422C02E215E023E040E00E94832FB8010E
:101B600086E096E00E9441208FEB91E01DC081301D
:101B700059F5C301B2010E94DB2C20912D04309154
:101B80002E0440912F04509130040E94F62D02E261
:101B900015E023E040E00E94832FB80186E096E044
:101BA0000E94412088EB91E09F938F93C8019F93FF
:101BB0000F930E941230B80186E096E00E946020E8
:101BC0000F900F900F900F908091FC039091FD0368
:101BD000892B09F440C06091FA057091FB05809152
:101BE000FC059091FD050E94DB2C20E030E04AE7E7
:101BF00054E40E94422C02E215E021E040E00E9401
:101C0000832FF80101900020E9F73197E252F54067
:101C100026E02E9FC0012F9F900D112464E770E0F5
:101C2000681B790B40E150E086E096E00E94F525C4
:101C3000B80186E096E00E94412085EB91E09F93F9
:101C40008F931F930F930E941230B80186E096E0A5
:101C50000E94602052C28091D904882351F002E290
:101C600015E020E040E06BA17CA1C1010E94832F20
:101C70000EC082EB91E09F938F9382E295E09F9359
:101C80008F930E9412300F900F900F900F90E2E20E
:101C9000F5E001900020E9F73197E252F54026E0A7
:101CA0002E9FC0012F9F900D11246AE770E0681BE2
:101CB000790B40E150E086E096E00E94F52562E273
:101CC00075E086E096E00E94412065E673E086E0DC
:101CD00096E00E94602015C2813009F0E9C160E001
:101CE00082E10E94F41D8091310490913204A0E0C1
:101CF000B0E084159505A605B70510F461E001C0B4
:101D000060E082E10E94F41DE12CF12C00E0A301CF
:101D100092016D897E898F89988D0E946004E2E02E
:101D2000EE2EE5E0FE2E80E2D7011D928A95E9F7BE
:101D300040E150E060E070E086E096E00E94F5252A
:101D400061E086E096E00E94FB2561E070E086E0BD
:101D500096E00E9401268091FC039091FD03892B5F
:101D600009F4EBC00E94A50320E030E040EF51E40D
:101D70000E94742B0E94AA2C161617067CF041E0D4
:101D800050E060E070E086E096E00E9407266AE39B
:101D900073E086E096E00E944120B3C1C301B20126
:101DA000B9EE4B16B3E05B066104710488F10E9442
:101DB000DB2C20E030E04AE754E40E94422C02E2AF
:101DC00015E021E040E00E94832F44E050E0B8019C
:101DD00082E095E00E94D92FF70101900020E9F7F9
:101DE000329780818E3209F4108262E075E086E0DD
:101DF00096E00E9441208CEA91E09F938F9382E2CB
:101E000095E09F938F930E94123062E275E017C0B5
:101E10000E94DB2C02E215E020E040E00E94832FCC
:101E2000B80186E096E00E94412087EA91E09F9306
:101E30008F93C8019F930F930E941230B80186E0E0
:101E400096E00E9441200F900F900F900F90C301D9
:101E5000B2010E94DB2C20912D0430912E04409180
:101E60002F04509130040E94F62D6B017C0120E07C
:101E700034E244E759E40E94EB2D1816F4F420E014
:101E800034E244E759E4C701B6010E94422C02E261
:101E900015E021E040E00E94832F45E050E0B801CA
:101EA00082E095E00E94D92F62E075E086E096E03E
:101EB0000E94412080EA91E037C020E030E44CE10C
:101EC00056E4C701B6010E94EB2D1816F4F420E089
:101ED00030E04AE754E4C701B6010E94422C02E216
:101EE00015E020E040E00E94832F45E050E0B8017B
:101EF00082E095E00E94D92F62E075E086E096E0EE
:101F00000E94412089E991E00FC002E215E020E043
:101F100040E0C701B6010E94832FB80186E096E039
:101F20000E94412083E991E09F938F93C8019F9382
:101F30000F930E941230B801DCC00E94A50320E07C
:101F400030E040EF51E40E94742B0E94AA2C161638
:101F500017060CF014CF8FE891E09F938F9372E2F5
:101F6000E72E75E0F72EFF92EF920E941230B70134
:101F700086E096E00E9441206091B0057091B10525
:101F80008091B2059091B3050E94DB2C2091290429
:101F900030912A0440912B0450912C040E94422C31
:101FA000870121E040E00E94832FB70186E096E0A0
:101FB0000E94412089E891E09F938F93FF92EF92D6
:101FC0000E941230B70186E096E00E94412085E829
:101FD00091E09F938F93FF92EF920E941230B7018E
:101FE00086E096E00E94412060910C0470910D04FF
:101FF00080910E0490910F040E94DB2C4B015C0138
:10200000609108047091090480910A0490910B0476
:102010000E94DB2C6D8B7E8B8F8B988F20E030E0C5
:1020200040E752E4C501B4010E94422C9B01AC017F
:102030006D897E898F89988D0E94422C2091290478
:1020400030912A0440912B0450912C040E94422C80
:102050006D8B7E8B8F8B988F20E030E041E655E4CE
:10206000C501B4010E94422C9B01AC016D897E899F
:102070008F89988D0E94F62D20E040E00E94832FEA
:10208000B70186E096E00E94412082E891E09F93AC
:102090008F93FF92EF920E941230B70186E096E094
:1020A0000E9441200FB6F894DEBF0FBECDBF29C0FD
:1020B00040E050E060E070E086E096E00E94F525A8
:1020C00062E086E096E00E94FB2541E050E060E09F
:1020D00070E086E096E00E94072685E791E09F93F6
:1020E0008F9382E295E09F938F930E94123062E279
:1020F00075E086E096E00E9441200F900F900F90CF
:102100000F908091E504882389F188891F928F932D
:1021100089891F928F938A891F928F938C891F922E
:102120008F938B891F928F938CE591E09F938F9370
:1021300082E295E09F938F930E94123048E150E035
:1021400060E070E086E096E00E94F52561E086E0C0
:1021500096E00E94FB2561E070E086E096E00E9438
:10216000012662E275E086E096E03CC048E150E07E
:1021700060E070E086E096E00E94F52561E086E090
:1021800096E00E94FB2541E050E060E070E086E0D0
:1021900096E00E94072686E491E09F938F9382E267
:1021A00095E09F938F930E94123062E275E086E083
:1021B00096E00E94412060E082E10E94F41DE2E48A
:1021C000F5E084E6DF011D928A95E9F78AE391E064
:1021D0009F938F93FF93EF930E94123062E475E018
:1021E00085E594E00E9460200FB6F894DEBF0FBE34
:1021F000CDBF0E94A50320E030E040EF51E40E94F3
:10220000742B0E94AA2C6B0177FD07C06930710501
:1022100034F068E0C62ED12C02C0C12CD12C8091A4
:1022200014048130F1F548E150E06CE570E086E09F
:1022300096E00E94F5258091310490913204A0E04F
:10224000B0E084159505A605B70518F461E273E0C2
:1022500002C064E273E086E096E00E944120E091D3
:102260000606F09107060684F785E02DEE24E39438
:10227000F12C07E010E02CE030E048E150E064E7AA
:1022800070E086E096E00995E0910606F091070679
:102290000088F189E02D03E010E096014AE150E06A
:1022A0003DC040E050E06CE570E086E096E00E94C2
:1022B000F5258091310490913204A0E0B0E08415BE
:1022C0009505A605B70518F461E273E002C064E263
:1022D00073E086E096E00E944120E0910606F091CE
:1022E00007060684F785E02DEE24E394F12C07E041
:1022F00010E02CE030E040E050E064E770E086E081
:1023000096E00995E0910606F09107060088F189AC
:10231000E02D03E010E0960142E050E066E770E057
:1023200086E096E0099586E096E00E944828809134
:10233000FC039091FD0321E082279093FD0380939D
:10234000FC0362E475E08AE496E00E9460208091DC
:10235000EC058823B1F080911404811112C086EE3F
:1023600094E00E94F22062E475E086EE94E00E9420
:10237000602007C08091E504882309F454CB61E014
:1023800053CBA496E2E10C94452F80912F069091B7
:102390003006A0913106B09132060196A11DB11D03
:1023A00080932F0690933006A0933106B0933206A7
:1023B000089580933B0690933C06409333065093D8
:1023C0003406609335067093360610922F061092ED
:1023D0003006109231061092320643E050E065EC70
:1023E00071E10E941E1C08950E94E21C6093370652
:1023F000709338068093390690933A0610922F0610
:102400001092300610923106109232060895CF9243
:10241000DF92EF92FF920F931F930E94E21CC090F5
:102420003706D0903806E0903906F0903A060091D1
:1024300033061091340620913506309136066C151E
:102440007D058E059F0588F0DC01CB018C199D0967
:10245000AE09BF0951E040E080179107A207B3071A
:1024600008F450E0852F942F10C0C094D094E094CD
:10247000F094C60ED71EE81EF91E81E090E0C0164B
:10248000D106E206F30608F480E01F910F91FF9059
:10249000EF90DF90CF90089560912F0670913006F5
:1024A00080913106909132060895EF92FF920F933A
:1024B0001F93FC017183608353834283358324839C
:1024C00017830683F186E0861F910F91FF90EF90AE
:1024D0000895EF92FF920F931F93CF93DF93EB0139
:1024E0007C012DE2E20EF11C49918C010F5F1F4F20
:1024F000BC0188E797E00E94AF230E151F0511F07D
:10250000C801F2CF8DE290E0CDB7DEB7E6E00C94E3
:10251000512FEF92FF920F931F93CF93DF937C0184
:102520008B01C0E0D0E0F80141918F01BE016E0D3A
:102530007F1D88E797E00E94AF232196C830D10520
:1025400091F788E090E0CDB7DEB7E6E00C94512F2C
:10255000EF92FF920F931F93CF93DF93EC01EA81E9
:10256000FB818DE2DF011D928A95E9F70A811B81CB
:1025700064EF71E07B01BFEFEB1AFB0A88E797E09D
:102580000E94AB23F80181938F01F1E2EF16F2E094
:10259000FF0611F0B701EECFEA81FB814081518146
:1025A000628173814D30504F6E4F7A4509F44EC0B1
:1025B0008DE2DF011D928A95E9F7EA81FB814DE00A
:1025C00050EF6EEF7AE54083518362837383178AFD
:1025D000168A89E083A38EE193E09F938F938A818B
:1025E0009B8184969F938F930E941230EA81FB8196
:1025F0008CE3808FEA81FB8140E050E067EA73E47E
:10260000418F528F638F748F40E050E064E172E439
:10261000458F568F678F70A384E690E093A782A7BB
:10262000BF0184EF91E00E946912EC81FD8188E096
:10263000DF011D928A95E9F76C817D8188EC90E03D
:102640000E9489120F900F900F900F90CDB7DEB7B8
:10265000E6E00C94512FA2E0B0E0E1E3F3E10C944A
:102660002D2F3C01DC018D919C9169837A830E941E
:10267000F220F30181858F9380858F937A817F93F8
:1026800069816F9381E193E09F938F9387818F930B
:1026900086818F930E941230D30116966D917C91A2
:1026A00017978D919C910E944120F3018081918127
:1026B000DC01ED91FC910190F081E02D6DE0099538
:1026C0000FB6F894DEBF0FBECDBFD3018D919C91A4
:1026D000DC01ED91FC910480F581E02D0995892BB9
:1026E000A1F3F30180819181DC01ED91FC910680E1
:1026F000F781E02D09958D3011F08A3031F7F30123
:102700004085518560E070E0868197810E94C22FEC
:1027100000E010E0A12CD3018D919C91DC01ED91A2
:10272000FC910480F581E02D0995892BB1F0FF24FF
:10273000F394FA0CF301068117810A0D111D8081B3
:102740009181DC01ED91FC910680F781E02D0995E6
:10275000F8018083AF2C00E010E061E070E080E0E1
:1027600090E00E94111D2A2D30E0D30118968D9122
:102770009C9119972817390729F470E0B12C88E04B
:10278000882E27C00F5F1F4F083EB3E01B071CF2C7
:10279000F4CF2D30B1F0492D50E0D30118962D9192
:1027A0003C9119974217530761F0292D622F671B3F
:1027B00099249394920EDC01A20FB11D2C912A3022
:1027C00041F7DF01A60FB11D1C92808181110CC061
:1027D000792D7A1508F0B6C1F30186819781FC0145
:1027E000E70FF11D272FE2CF833291F3633080F39F
:1027F00080E07F01E80EF11CD7019C91903221F41A
:102800008F5F8613F6CFE4CF9930D1F3861701F3AB
:10281000DF01A80FB11D9C919D3339F0903211F06A
:10282000993009F41C928F5FF1CF861789F28F5F80
:102830001C928F01080F111DD8019C91903221F438
:102840008F5F8613F6CFC4CF9930D1F3861709F482
:10285000BFCF60E573E0C7010E94C92F892B19F52E
:10286000C8010E94A42FBC01882777FD8095982F6E
:102870000E94DD2C6B017C01F301028113819B011D
:10288000AC01D80159966D917D918D919C915C9789
:102890000E943B2C882309F49BCFF801C18ED28E75
:1028A000E38EF48E30C165E573E0C7010E94C92F45
:1028B000892B29F5C8010E94A42FBC01882777FD28
:1028C0008095982F0E94DD2C6B017C01D30112961C
:1028D0000D911C9113979B01AC01F801658D768DCC
:1028E000878D90A10E943B2C882309F471CFD801D9
:1028F0005D96CD92DD92ED92FC92909704C16AE5CF
:1029000073E0C7010E94C92F892B39F4F301E280DB
:10291000F380F6E0EF0EF11C72C06DE573E0C701C5
:102920000E94C92F892B91F4D3011296ED90FC904F
:102930001397C8010E94A42FF70126893789281709
:10294000390709F445CF978B868BDDC061E673E0CC
:10295000C7010E94C92F892B89F4D3011296ED90EB
:10296000FC901397C8010E94A42FF701248130E046
:102970002817390709F42CCF8483C5C064E673E0B7
:10298000C7010E94C92F892B89F4D3011296ED90BB
:10299000FC901397C8010E94A42FF701258130E015
:1029A0002817390709F414CF8583ADC067E673E0B3
:1029B000C7010E94C92F892B91F4D3011296ED9083
:1029C000FC901397C8010E94A42FF70121A132A106
:1029D0002817390709F4FCCE92A381A394C06AE6B4
:1029E00073E0C7010E94C92F892BA9F4D80113965F
:1029F0001C92F301E280F380F4E2EF0EF11CB801C7
:102A0000C7010E94C92F892B09F4E2CEB801C70182
:102A10000E94D22F78C06DE673E0C7010E94C92FD3
:102A2000892B89F4D3011296ED90FC901397C8017D
:102A30000E94A42FF70123A130E02817390709F4D9
:102A4000C7CE83A360C060E773E0C7010E94C92FAF
:102A5000892B89F4D3011296ED90FC901397C8014D
:102A60000E94A42FF70120A530E02817390709F4A8
:102A7000AFCE80A748C063E773E0C7010E94C92FAB
:102A8000892B89F4D3011296ED90FC901397C8011D
:102A90000E94A42FF70121A530E02817390709F477
:102AA00097CE81A730C066E773E0C7010E94C92FA7
:102AB000892B91F4D3011296ED90FC901397C801E5
:102AC0000E94A42FF70122A533A52817390709F47E
:102AD0007FCE93A782A717C069E773E0C7010E9462
:102AE000C92F892B99F4D3011296ED90FC9013977E
:102AF000C8010E94A42FF70124A530E02817390748
:102B000009F466CE84A7BB24B39462CE6CE773E06D
:102B1000C7010E94C92F892B09F05ACED301149600
:102B2000ED91FC911597DF01882D1D928A95E9F7AB
:102B3000D30114966D917C91159788EC90E00E94DA
:102B4000891246CEBB2039F0F3016281738184EF94
:102B500091E00E9469122296EEE00C94492F0F93A7
:102B60001F93FC01862F0FEF1FEF98010083118345
:102B70002283338310861186128613864FEF59EC19
:102B80006AE97BE3408B518B628B738B408F518F53
:102B9000628F738F40A351A362A373A340A751A771
:102BA00062A773A740AB51AB62AB73AB00AF11AF81
:102BB00022AF33AFDF01A05CBF4F4FEF50E0119663
:102BC0005C934E9314960D931D932D933C93139702
:102BD00018960D931D932D933C93139718961C9262
:102BE00011961C92509692E09C9311961C9211960D
:102BF0001C9211961C9212961D921D921D921C926F
:102C00001397149611961C921E92129611961C926E
:102C10001E925A971C92E759FF4F80831F910F9184
:102C200008952FEB260F862F90E0263010F4C797DB
:102C300008956156663018F4875591090895C09734
:102C40000895CF93FB0160E070E0CB01C19120EDCE
:102C50002C0F2A3078F4AAE0B0E09B01AC010E946E
:102C6000162F6C0F711D811D911D60537109810913
:102C70009109ECCFCF9108950F931F93CF93FC014F
:102C8000EA5AFF4FC1E020812D3219F0C0E08F01D8
:102C900003C08C01095A1F4FB8010E9421169B01E5
:102CA000AC01A4E6B0E00E94162FF801DF012191EB
:102CB00030ED320F3A30D0F32E3249F511962C9187
:102CC000119730ED320F3A3010F530E020533109D2
:102CD0004AE0429F8001439F100D1124222717FDD7
:102CE0002095322F600F711F821F931F12960C9137
:102CF00020ED200F2A3058F410E00053110922274C
:102D000017FD2095322F600F711F821F931FCC2358
:102D100039F090958095709561957F4F8F4F9F4FBB
:102D2000CF911F910F9108954F925F926F927F9272
:102D30008F929F92AF92BF92CF92DF92EF92FF92CB
:102D4000CF93DF93EC01CA5ADF4FBE010E942116D8
:102D50002B013C0124E630E040E050E00E94EE2EE2
:102D60009B01AC0160EA76E881E090E00E94CA2E07
:102D70006B017C01FE01819190ED980F9A30D8F3A0
:102D80008E3209F5EF0180E1882E87E2982EA12C82
:102D9000B12CA99180ED8A0F8A30A8F4B0E0D097C9
:102DA000A50194010E94212FC60ED71EE81EF91E10
:102DB000C501B4012AE030E040E050E00E94EE2E70
:102DC00049015A01E6CFC701B6016B5F7F4F8F4FB4
:102DD0009F4F26E030E040E050E00E94EE2E690177
:102DE0007A01C301B20124E630E040E050E00E94E5
:102DF000EE2E60E472E48FE090E00E94CA2EC60ED0
:102E0000D71EE81EF91EC701B601DF91CF91FF90D2
:102E1000EF90DF90CF90BF90AF909F908F907F907A
:102E20006F905F904F9008954F925F926F927F9254
:102E30008F929F92AF92BF92CF92DF92EF92FF92CA
:102E4000CF93DF93EC01CA5ADF4FBE010E942116D7
:102E50002B013C01FE01819190ED980F9A30D8F33F
:102E60008E3221F5EF0190E1892E97E2992EA12C67
:102E7000B12CC12CD12C7601A99180ED8A0F8A301A
:102E8000C0F4B0E0D097A50194010E94212FC60E96
:102E9000D71EE81EF91EC501B4012AE030E040E06B
:102EA00050E00E94EE2E49015A01E6CFC12CD12CF0
:102EB0007601A301920160EA76E881E090E00E9449
:102EC000CA2E6C0D7D1D8E1D9F1DDF91CF91FF9031
:102ED000EF90DF90CF90BF90AF909F908F907F90BA
:102EE0006F905F904F900895DB01FA018D918823D8
:102EF00019F091918917D1F390E00895CF92DF9264
:102F0000EF92FF921F93CF93DF93EC01FC01EB5AFA
:102F1000FF4F1081112309F4D7C0319660810E94C0
:102F20001116182FFE01E95AFF4F6081CE010E9451
:102F3000111640E1149F800D1124FE01EC5AFF4F41
:102F400090818913B9C074961081112309F485C04A
:102F5000369680819181019691838083B697808196
:102F60009181A281B381349780839183A283B383BB
:102F70003C9680819181A281B38134978083918333
:102F8000A283B383799680818823A1F1813009F0EF
:102F90007EC18C819D81AE81BF8188839983AA8304
:102FA000BB838C859D85AE85BF8588879987AA87D9
:102FB000BB878C899D89AE89BF89888B998BAA8BA9
:102FC000BB8B8C8D9D8DAE8DBF8D888F998FAA8F79
:102FD000BB8F8CA59DA5AEA5BFA588A799A7AAA7BD
:102FE000BBA78CA99DA9AEA9BFA988AB99ABAAAB79
:102FF000BBAB4DC18CA19DA1AEA1BFA188A399A3DC
:10300000AAA3BBA38C819D81AE81BF818883998354
:10301000AA83BB838C899D89AE89BF89888B998B54
:10302000AA8BBB8B8C8D9D8DAE8DBF8D888F998F1C
:10303000AA8FBB8FFE01E05CFF4FDE01AE5BBF4F8E
:103040008D919C91918380838CAD9DADAEADBFADD4
:1030500088AF99AFAAAFBBAF1AC14C815D816E81B9
:103060007F81411551056105710509F410C1FE010B
:10307000E85BFF4F80819181A281B3813497808387
:103080009183A283B383B1968081882381F08130BC
:1030900009F0FDC0488359836A837B838C859D85B5
:1030A000AE85BF8588879987AA87BB87F0C048838C
:1030B00059836A837B83EBC0C059DF4F8881998134
:1030C00001969983888396C0FC01EA59FF4F3081AD
:1030D0008B599F4F7C0131111DC06E0196E5C90EC1
:1030E000D11C41E853E0B601CE010E947417892B30
:1030F00011F481E00CC047E853E0B601CE010E9414
:103100007417892B19F4F7011082C1C082E0D7012E
:103110008C93BDC0DC01EC91E23009F4B8C0CE0163
:103120008A5A9F4FDC012C91222309F4B0C0B0E2EF
:10313000EB9FF0011124E32B3197E932F10508F000
:10314000A6C0EC5CFF4F0C94102FCE010E943C16E1
:103150006C837D838E839F830E94E21CC85BDF4F5C
:103160001CC0C859DF4F81E0213409F076C076C019
:10317000FE01E759FF4F8081882321F0CE010E9494
:10318000141703C0CE010E9494166C8B7D8B8E8B1E
:103190009F8B0E94E21CC05BDF4F688379838A8328
:1031A0009B8375C0233509F072C08C899D89AE89D7
:1031B000BF89B095A095909581959F4FAF4FBF4F18
:1031C0008C8B9D8BAE8BBF8B62C0FE01E759FF4F8E
:1031D0008081882341F0CE010E9414176C8F7D8F6F
:1031E0008E8F9F8F54C0CE010E9494166C8F7D8F5E
:1031F0008E8F9F8F10E04BC0273509F048C08C8D13
:103200009D8DAE8DBF8DB095A095909581959F4F6A
:10321000AF4FBF4F8C8F9D8FAE8FBF8F38C0CE0109
:103220000E943C166CA77DA78EA79FA730C0CE0139
:103230000E943C166CAB7DAB8EAB9FAB28C0BC0133
:10324000CE010E9421166C877D878E879F871FC0C5
:10325000C859DF4F81E0213308F480E0888317C02C
:103260000E94A42FCE5BDF4F9927998388830FC0DC
:10327000CE010E943C166CAF7DAF8EAF9FAF07C0F2
:10328000CE010E943C166CA37DA38EA39FA3812F29
:10329000DF91CF911F91FF90EF90DF90CF90089535
:1032A000A1E0B0E0E6E5F9E10C94332F6C01262FA4
:1032B000FC01E659FF4F40815181628173814F5F6C
:1032C0005F4F6F4F7F4F40835183628373838C01C5
:1032D00009591F4F8B5A9F4F7C01243281F128F4EA
:1032E0002A3069F02D30E9F50AC02A3241F02C323B
:1032F000C1F5F601EC5AFF4F808182278083F801E7
:1033000080818F3060F4F601E80FF11DEA5AFF4F1B
:103310001082C60129830E947E17298101C080E0A6
:10332000F601EA59FF4F90819F5F9083F801108268
:1033300091E02A3209F090E0F70190832AC0F80169
:103340001082F601EA59FF4F10827297108271962F
:1033500082E08083F7011082F601E859FF4F108266
:1033600017C0F80180818E3048F491E0980F908367
:10337000F601E80FF11DEA5AFF4F2083F701808123
:10338000811106C0F601EC5AFF4F808182278083AD
:1033900080E02196E8E00C944F2FA0E1B0E0E3ED4F
:1033A000F9E10C942B2F69837A838B839C83CA0168
:1033B000B90127013801A60195010E94742B25E36C
:1033C0003AEF4EE85CE30E94F62D6B017C010E940F
:1033D000592E6D877E878F87988BC701B6010E9413
:1033E0003F2C6D837E838F83988725E33AEF4EE8E9
:1033F0005CE369817A818B819C810E94F62D6B014F
:103400007C0125E33AEF4EE85CE3C301B2010E9480
:10341000F62D2B013C01C701B6010E94592E4B012C
:103420005C01C701B6010E943F2C69837A838B83BC
:103430009C83C301B2010E94592E69877A878B87CA
:103440009C87C301B2010E943F2C6B017C0129853E
:103450003A854B855C8569817A818B819C810E944C
:10346000F62D2B013C01A7019601C501B4010E9474
:10347000F62D2D813E814F8158850E94F62D9B01AE
:10348000AC01C301B2010E94742B9B01AC010E94EC
:10349000F62D2B013C012D853E854F855889C701AE
:1034A000B6010E94F62D9B01AC010E94F62D9B01F6
:1034B000AC01C301B2010E94752B0E94632E2B0147
:1034C0003C0129853A854B855C85C501B4010E9484
:1034D000F62D4B015C01A701960169817A818B81F0
:1034E0009C810E94F62D2D813E814F8158850E943E
:1034F000F62D9B01AC01C501B4010E94752B9B0107
:10350000AC01C301B2010E94E82B26E73BE742EC85
:103510005AE40E94F62D6096E0E10C94472FA0E05B
:10352000B0E0E5E9FAE10C94332FE901611571058A
:1035300051F0FC01C088D188E288F388FB01C08289
:10354000D182E282F3824115510551F0FC01C08C19
:10355000D18CE28CF38CFA01C082D182E282F382B8
:10356000209701F18C01045B1F4FF801808191814C
:10357000A281B3818F3F9F4FAF4FBF4F61F00E9439
:10358000E21CF8010081118122813381601B710BE3
:10359000820B930B03C06FEF7FEFCB0168837983BE
:1035A0008A839B83CDB7DEB7E8E00C944F2FA0E071
:1035B000B0E0EDEDFAE10C94332FE90161157105EE
:1035C00051F0FC01C084D184E284F384FB01C08209
:1035D000D182E282F3824115510551F0FC01C08095
:1035E000D180E280F380FA01C082D182E282F3824C
:1035F000209701F18C010C5B1F4FF80180819181B4
:10360000A281B3818F3F9F4FAF4FBF4F61F00E94A8
:10361000E21CF8010081118122813381601B710B52
:10362000820B930B03C06FEF7FEFCB01688379832D
:103630008A839B83CDB7DEB7E8E00C944F2FAAE0D6
:10364000B0E0E5E2FBE10C94292F2B015A87498772
:1036500019019401AE014F5F5F4FBE016B5F7F4F59
:103660000E94D71A41145104B9F06D817E818F8177
:10367000988524E630E040E050E00E94EE2E61356F
:1036800071051CF02CE637E002C020ED37E0620F38
:10369000731FF2017183608389859A85892BB1F04C
:1036A0006D817E818F81988544E6442E512C612C5A
:1036B000712CA30192010E94EE2ECA01B901A3014F
:1036C00092010E94EE2EE985FA856083211431046F
:1036D00061F06D817E818F81988520E137E240E045
:1036E00050E00E94EE2EF10120830115110561F0DA
:1036F00069817A818B819C8120E432E44FE050E043
:103700000E94EE2EF8012083E114F104A1F06981FA
:103710007A818B819C8120E137E240E050E00E9479
:10372000EE2ECA01B90124E630E040E050E00E94EC
:10373000EE2EF7016083C114D104A9F069817A816A
:103740008B819C8134E6432E512C612C712CA3017A
:1037500092010E94EE2ECA01B901A30192010E94BA
:10376000EE2EF6016083A114B10461F069817A81C3
:103770008B819C8124E630E040E050E00E94EE2EF8
:10378000F50160832A96E2E10C94452FFC0160A1CB
:1037900071A182A193A16F3FF9EC7F07FAE98F072E
:1037A000FBE39F0749F00E94DD2C20E030E048EC6D
:1037B00052E40E94422C089560E074E284E799E4A8
:1037C0000895FC0160A571A582A593A56F3FF9EC52
:1037D0007F07FAE98F07FBE39F0749F00E94DB2C84
:1037E00020E030E048EC52E40E94422C089560E072
:1037F00070E080E89FEB0895CF92DF92EF92FF9206
:103800000E94E11B6B017C0120E030E040E85FEBAF
:103810000E943B2C882349F026E53EE04DEE5FE315
:10382000C701B6010E94F62D04C060E070E080E898
:103830009FEBFF90EF90DF90CF9008958230E8F4F7
:10384000E82FF0E0EE0FFF1FE35CF94F7183608318
:10385000813041F0809169008C7F842B80936900D6
:10386000E89A089580916900440F551F440F551F31
:10387000837F842B80936900E99A08951F920F92A9
:103880000FB60F9211242F933F934F935F936F9333
:103890007F938F939F93AF93BF93EF93FF93809109
:1038A0003D0690913E06892B29F0E0913D06F0916E
:1038B0003E060995FF91EF91BF91AF919F918F9136
:1038C0007F916F915F914F913F912F910F900FBE1C
:1038D0000F901F9018951F920F920FB60F92112400
:1038E0002F933F934F935F936F937F938F939F9308
:1038F000AF93BF93EF93FF9380913F069091400663
:10390000892B29F0E0913F06F09140060995FF913F
:10391000EF91BF91AF919F918F917F916F915F9147
:103920004F913F912F910F900FBE0F901F901895C0
:103930001F920F920FB60F9211242F933F938F93E4
:103940009F93AF93BF938091420690914306A091BD
:103950004406B09145063091410626E0230F2D37ED
:1039600020F40296A11DB11D05C029E8230F03967E
:10397000A11DB11D209341068093420690934306FA
:10398000A0934406B0934506809146069091470661
:10399000A0914806B09149060196A11DB11D8093E2
:1039A000460690934706A0934806B0934906BF91F8
:1039B000AF919F918F913F912F910F900FBE0F90DC
:1039C0001F9018952FB7F8946091420670914306A6
:1039D00080914406909145062FBF08953FB7F89413
:1039E0008091460690914706A0914806B0914906FD
:1039F00026B5A89B05C02F3F19F00196A11DB11D4A
:103A00003FBF6627782F892F9A2F620F711D811D66
:103A1000911D43E0660F771F881F991F4A95D1F7C4
:103A20000895CF92DF92EF92FF92CF93DF936B01D5
:103A30007C010E94EE1CEB01C114D104E104F104ED
:103A400079F00E94EE1C6C1B7D0B683E7340A0F366
:103A500081E0C81AD108E108F108C851DC4FECCF69
:103A6000DF91CF91FF90EF90DF90CF900895789401
:103A700084B5826084BD84B5816084BD85B5826073
:103A800085BD85B5816085BDEEE6F0E08081816011
:103A90008083E1E8F0E01082808182608083808111
:103AA00081608083E0E8F0E0808181608083E1EBE9
:103AB000F0E0808184608083E0EBF0E080818160D1
:103AC0008083EAE7F0E08081846080838081826087
:103AD0008083808181608083808180688083109270
:103AE000C10008958093090108958E3008F08E502A
:103AF00087702091090190E4299F90011124822B65
:103B000080937C0080917A00806480937A00809119
:103B10007A0086FDFCCF809178002091790090E0BA
:103B2000922B0895833081F028F4813099F082300F
:103B3000A1F008958630A9F08730B9F08430D1F42F
:103B4000809180008F7D03C0809180008F7780936B
:103B50008000089584B58F7702C084B58F7D84BDC1
:103B600008958091B0008F7703C08091B0008F7D61
:103B70008093B0000895CF93DF9390E0FC01EA5C5E
:103B8000FC4F2491FC01E65BFC4F8491882349F1B2
:103B900090E0880F991FFC01EE58FC4FA591B4915D
:103BA00088599C4FFC01C591D4919FB7611108C001
:103BB000F8948C91209582238C93888182230AC06B
:103BC000623051F4F8948C91322F309583238C938A
:103BD0008881822B888304C0F8948C91822B8C93EB
:103BE0009FBFDF91CF910895A1E0B0E0EAEFFDE142
:103BF0000C94372F282F30E0F901EE5DFC4F8491B3
:103C0000F901EA5CFC4F1491F901E65BFC4F049169
:103C10000023C9F0882321F069830E94921D6981E5
:103C2000E02FF0E0EE0FFF1FE859FC4FA591B49193
:103C30009FB7F8948C91611103C01095812301C046
:103C4000812B8C939FBF2196E4E00C94532FFC01B1
:103C500024853585F901E05CFF4F808191813296A2
:103C600020813181821B930B8F7399270895FC016A
:103C700084859585FC01E05CFF4F4081518132963F
:103C8000208131814217530741F00190F081E02DEE
:103C9000E80FF91F808190E008958FEF9FEF08955E
:103CA000FC0184859585FC01E05CFF4F40815181DA
:103CB0003296208131814217530779F0A081B1817A
:103CC000A80FB91F8C91208131812F5F3F4F2F7337
:103CD00033273183208390E008958FEF9FEF08957D
:103CE000FC0181A1882329F0A489B5898C9186FFE4
:103CF000FBCF11A20895CF93DF93FC012685378572
:103D0000D901A05CBF4F8D919C91119701968F7343
:103D10009927E901CE5BDF4F4881598184179507C8
:103D2000D9F30D90BC91A02DA20FB31F6C93A68563
:103D3000B785A05CBF4F11969C938E93A689B789D7
:103D40002C9181E090E0078C02C0880F991F0A94A3
:103D5000E2F7282B2C9381E081A30488F589E02DDC
:103D600080818064808381E090E0DF91CF9108952D
:103D700008951F920F920FB60F9211242F933F9325
:103D80004F938F939F93EF93FF938091C00082FD99
:103D90001CC04091C6008091F0069091F1060196FA
:103DA0008F7399272091F2063091F30682179307BB
:103DB00071F0E091F006F091F106E055F94F408383
:103DC0009093F1068093F00602C08091C600FF91A7
:103DD000EF919F918F914F913F912F910F900FBE37
:103DE0000F901F9018958AE496E00E94271E892B59
:103DF00011F00E94B81E08951F920F920FB60F92F5
:103E000011242F933F938F939F93EF93FF932091D0
:103E1000AC063091AD068091AE069091AF062817A2
:103E2000390731F48091C1008F7D8093C10014C0A7
:103E3000E091AE06F091AF06E459F94F20818091F0
:103E4000AE069091AF0601968F7399279093AF06B7
:103E50008093AE062093C600FF91EF919F918F91C2
:103E60003F912F910F900FBE0F901F901895CF92FA
:103E7000DF92EF92FF92CF93DF93EC016A017B0117
